:100000009E28A40044200C080D040319992893206D
:1000100084132408800664000D280E288C0A031916
:100020008D0F0B28800699288F002608840024094C
:10003000452084138F0803199928F03091000E0889
:1000400080389000F03091030319910003198F0359
:10005000031999280C0892000D089300273064209A
:1000600012088C0013088D00482003010C18240886
:100070008E1F24088E0803190301900F4128800663
:100080001F28422800002228FF3A8417800599285B
:100090000D080C0403198C0A80300C1A8D060C19FB
:1000A0008D068C188D060D0D8C0D8D0D99288F01E8
:1000B0008E00FF308E07031C8F07031C9928033026
:1000C0008D00E630652059288D01FC3E8C008D099D
:1000D000031C7028FF3000008C0703186B288C0766
:1000E00064008D0F6A2808008D018F018E00023098
:1000F0007C288E0001307C2894000F080D02031D1F
:1001000083280E080C020430031801300319023052
:100110001405031DFF3099280038031DFF30040526
:10012000031DFF3099288C098D098C0A03198D0A4B
:100130000800831303138312640008008316F4304D
:10014000850015308600831286118316861183126E
:100150008511831685118312AC01AD01AA01AB0193
:10016000DD2185148316851083128614831686106C
:1001700064008312051DF42A07308F00D030582008
:1001800086108316861083128614831686108312B7
:100190000130A800A90128088C0029088D008F01D2
:1001A000FA307920031DE428861583168611023063
:1001B000831264208611831686110D308312642009
:1001C000A80A0319A90FCB280030061901308C00AA
:1001D000003074209E000030061A01308C00003080
:1001E0007420A0001E08840020088C20031D4029D4
:1001F0006400061EAB296400061D7929861083164B
:100200008610831285148316851083120130A8008E
:10021000A90128088C0029088D008F01143079204D
:10022000031D3429051083160510831210308C002D
:1002300003308D00053084000130012086128316C2
:1002400086128312F4308C0002308D000630840058
:1002500020300120143057206400061A3029EE2A7D
:10026000A80A0319A90F0929061383160613831276
:10027000AA0A640029302A02031C3F29192AC4282B
:10028000AA01DD210C22851483168510831201300A
:10029000A800A90128088C0029088D008F010F30C3
:1002A0007920031D71290510831605108312ED3086
:1002B0008C0002308D000530840001300120861250
:1002C00083168612831217308C0003308D0006309F
:1002D00084002030012014305720A80A0319A90FE8
:1002E0004A29AC0A640009302C02031C78297929B8
:1002F000C428AA010530AC0085148316851083122A
:100300000130A800A90128088C0029088D008F0160
:1003100014307920031DAA290510831605108312B5
:1003200010308C0003308D00053084000130012036
:1003300086128316861283121C308C0003308D00C7
:10034000063084002030012014305720A80A0319F9
:10035000A90F8329C428AA010230AC008514831692
:10036000851083120130A800A90128088C002908F3
:100370008D008F0114307920031DDC2905108316B0
:1003800005108312E8308C0002308D0005308400A7
:10039000013001208612831686128312F4308C00FD
:1003A00002308D00063084002030012014305720A8
:1003B000A80A0319A90FB529C4280130A800A9016A
:1003C00028088C0029088D008F0105307920031D35
:1003D000072A0510831605108312FC308C000230AA
:1003E0008D000530840001300120861283168612AC
:1003F000831208308C0003308D00063084002030DA
:10040000012014305720A80A0319A90FE0298510EC
:1004100083168510831208000630A6008030A400E1
:100420004B308E000A3014206E308E000A301420BB
:100430000800AD01AC01DD21AA01AD0A86148316C6
:100440008610831285158316851183120130A8004A
:10045000A90128088C0029088D008F01143079200B
:10046000031D3F2A6400051E732A0A305720861098
:10047000831686108312A80A0319A90F292A851149
:10048000831685118312851483168510831201301B
:10049000A800A90128088C0029088D008F010A30C6
:1004A0007920031D6D2A10308C0003308D0005303B
:1004B00084000130012086128316861283121C30BC
:1004C0008C0003308D000630840020300120143071
:1004D0005720A80A0319A90F4A2A640011302D02D7
:1004E00003187C2A1B2A01308F00F4305820851114
:1004F0008316851183120229AD01DD21AD0A0B306F
:100500008F00B8305820861483168610643083120A
:10051000572086108316861083120130A800A90187
:1005200028088C0029088D0001308F00F4307920D4
:10053000031DB72A6400061CA12A0617831606139A
:1005400083126400061CA52AAB016400061CA92ABC
:10055000C4286400051AAD2A732A861083168610F3
:100560000A3083125720A80A0319A90F902A85146C
:100570008316851083120130A800A90128088C0079
:1005800029088D008F011E307920031DE12AE830F3
:100590008C0002308D00053084000130012086126D
:1005A000831686128312F4308C0002308D000630E0
:1005B00084002030012014305720A80A0319A90F05
:1005C000BE2AAB0A640013302B020318F42A64001D
:1005D00006302D02031CED2AC4287D2A0C2201308E
:1005E0008F00F430582079298510831685108312E6
:1005F0008610831686108312851583168511831243
:1006000007308F00D0305820851183168511831252
:10061000AC0A640005302C020318B12864000618E7
:10062000F42A6400051D182B6400061EB1280E2B49
:100630006400061EB1286400061C182B861483165D
:100640008610831203308F00E830582086108316FE
:0A06500086108312182B63002B2B79
:02400E00F53F7C
:00000001FF
